S01A000064656D6F70726F675F73746D3332663736372E737265638B
S3150800800000000820FD8C0008C98C0008CB8C0008ED
S31508008010CD8C0008CF8C0008D18C00080000000029
S31508008020000000000000000000000000D38C0008DB
S31508008030D58C000800000000D78C0008D98C0008F1
S315080080404D8D00084D8D00084D8D00084D8D00089A
S315080080504D8D00084D8D00084D8D00084D8D00088A
S315080080604D8D00084D8D00084D8D00084D8D00087A
S315080080704D8D00084D8D00084D8D00084D8D00086A
S315080080804D8D00084D8D00084D8D00084D8D00085A
S315080080904D8D00084D8D00084D8D00084D8D00084A
S315080080A04D8D00084D8D00084D8D00084D8D00083A
S315080080B04D8D00084D8D00084D8D00084D8D00082A
S315080080C04D8D00084D8D00084D8D00084D8D00081A
S315080080D04D8D00084D8D00084D8D00084D8D00080A
S315080080E04D8D00084D8D00084D8D00084D8D0008FA
S315080080F04D8D00084D8D00084D8D00084D8D0008EA
S315080081004D8D00084D8D00084D8D00084D8D0008D9
S315080081104D8D00084D8D00084D8D00084D8D0008C9
S315080081204D8D00084D8D00084D8D00084D8D0008B9
S315080081304D8D00084D8D00084D8D00084D8D0008A9
S315080081404D8D00084D8D00084D8D00084D8D000899
S315080081504D8D00084D8D00084D8D00084D8D000889
S315080081604D8D00084D8D00084D8D00084D8D000879
S315080081704D8D00084D8D00084D8D0008000000004B
S315080081804D8D00084D8D00084D8D00084D8D000859
S315080081904D8D00084D8D00084D8D00084D8D000849
S315080081A04D8D00084D8D00084D8D00084D8D000839
S315080081B04D8D00084D8D00084D8D00084D8D000829
S315080081C04D8D00084D8D0008000000004D8D0008FB
S315080081D04D8D00084D8D00084D8D00084D8D000809
S315080081E04D8D00084D8D00084D8D00084D8D0008F9
S311080081F04D8D00084D8D0008EE11AA55B3
S315080081FC10B5054C237833B9044B13B10448AFF3C7
S3150800820C00800123237010BD4C00002000000000E4
S3150800821C48C6000808B5034B1BB103490348AFF31E
S3150800822C008008BD000000005000002048C6000869
S3150800823C53B94AB9002908BF00281CBF4FF0FF31B3
S3150800824C4FF0FF3000F072B9ADF1080C6DE904CEB1
S3150800825C00F006F8DDF804E0DDE9022304B0704707
S3150800826C2DE9F047089E04468846002B4BD18A42D6
S3150800827C154667D9B2FA82F24AB1C2F1200701FA59
S3150800828C02F320FA07F7954047EA030894404FEAA9
S3150800829C154E230CB8FBFEF71FFA85FC0EFB178848
S315080082AC43EA084307FB0CF1994209D9EB1807F185
S315080082BCFF3080F01B81994240F21881023F2B4413
S315080082CC5B1AA4B2B3FBFEF00EFB103344EA03446C
S315080082DC00FB0CFCA44509D92C1900F1FF3380F0DE
S315080082EC0781A44540F2048102382C4440EA074031
S315080082FCA4EB0C0400271EB1D4400023C6E90043A6
S3150800830C3946BDE8F0878B4209D9002E00F0EB8080
S3150800831C0027C6E9000138463946BDE8F087B3FAA6
S3150800832C83F7002F47D18B4202D3824200F2FA80A0
S3150800833C841A61EB030301209846002EE0D0C6E9A7
S3150800834C0048DDE702B9FFDEB2FA82F2002A40F0F5
S3150800835C8F80491B4FEA154E1FFA85F80127B1FB8A
S3150800836CFEFC230C0EFB1C1143EA014308FB0CF123
S3150800837C994207D9EB180CF1FF3002D2994200F258
S3150800838CCD808446591AA3B2B1FBFEF00EFB10142D
S3150800839C43EA044408FB00F8A04507D92C1900F158
S315080083ACFF3302D2A04500F2B6801846A4EB0804A7
S315080083BC40EA0C409FE7C7F1200CBB4022FA0CFEA2
S315080083CC4EEA030E01FA07F420FA0CF521FA0CF31F
S315080083DC4FEA1E482543B3FBF8F92C0C08FB193356
S315080083EC1FFA8EFA44EA034309FB0AF49C4202FA82
S315080083FC07F200FA07F10BD91EEB030309F1FF305C
S3150800840C80F087809C4240F28480A9F1020973446B
S3150800841C1B1BADB2B3FBF8F008FB103345EA03445B
S3150800842C00FB0AFAA24508D91EEB040400F1FF3337
S3150800843C6BD2A24569D90238744440EA0940A0FBBC
S3150800844C0289A4EB0A044C45C2464B4654D351D078
S3150800845C002E69D0B1EB0A0564EB030404FA0CFC94
S3150800846CFD40FC404CEA0505C6E90054002747E7E1
S3150800847CC2F1200320FA03F7954001FA02F021FA1B
S3150800848C03F34FEA154E3843010CB3FBFEF71FFAFC
S3150800849C85F80EFB173341EA034107FB08F38B42B9
S315080084AC04FA02F407D9691807F1FF3C2FD28B425C
S315080084BC2DD9023F2944CB1A81B2B3FBFEF00EFB31
S315080084CC103341EA034100FB08F38B4207D96918BC
S315080084DC00F1FF3C17D28B4215D902382944C91A28
S315080084EC40EA07473BE73746304609E70746E7E6DB
S315080084FC1846FBE64145ABD2B8EB020A69EB0E020D
S3150800850C01381346A4E76046E9E7184695E7674637
S3150800851CD1E781467CE702382C4447E7ACF1020CDC
S3150800852C2B442FE7384608E73746E9E6704700BF7D
S3150800853C08B500F023FA00F09FF800F0F3F900F004
S3150800854CCBF800F033F80021084600F003FA08BD12
S3150800855C08B500F09BF800F019F900F089F808BD89
S3150800856C08B50948094B03604FF46143436000237F
S3150800857C8360C36003610C2242618361C361036239
S3150800858C436202F05DFB08BD68000020004800400D
S3150800859C08B5002301220146034802F08AFA08B1FD
S315080085AC002008BD0120FCE76800002008B5FFF78D
S315080085BCD7FF08BDBFF34F8F0549CA6802F4E062BE
S315080085CC044B1343CB60BFF34F8F00BFFDE700BFCF
S315080085DC00ED00E00400FA0508B5214B1B78B3B989
S315080085EC2048FFF7D5FF012800D008BD1D4B1B7886
S315080085FC013BDBB23F2BF8D800F0C1F91A4B1860D7
S3150800860C174B01221A70194B00221A70EDE7174BFB
S3150800861C1B78013313481844FFF7BAFF012813D106
S3150800862C124A13780133DBB213700E4A127893424E
S3150800863CDBD10B4A002111700A4A5278FF2AD4D191
S3150800864C022BD2D1FFF7B6FF00F099F9064B1B683F
S3150800865C64339842C9D9024B00221A70C5E700BF89
S3150800866C29010020E80000202C0100202A01002006
S3150800867C08B5FFF7B1FF08BD08B5002280210248EE
S3150800868C01F0FEF808BD00BF0004024010B500F06A
S3150800869C76F90E4B1B68C31AB3F5FA7F0CD304464E
S315080086AC0B4B1B784BB90122094B1A7080210948D0
S315080086BC01F0E6F8054B1C6010BD0022044B1A703D
S315080086CC8021044801F0DCF8F4E700BF34010020EF
S315080086DC300100200004024010B502F0E7FA00F061
S315080086EC4EF900F5FA70134B186000F048F942F28F
S315080086FC10730344104A136002F082FE0F4A0023DB
S3150800870C138053800E4A138053800E4A138053806D
S3150800871C4EF6030002F0B4FE02F004FB0A4C2046A7
S3150800872C02F014FB0621204602F0A2FC02F0BEFC65
S3150800873C10BD00BF4401002038010020B8330020CA
S3150800874CB4330020B03300203C01002008B50C4B94
S3150800875C1B7813F0400F09D113F0020F06D0094B02
S3150800876C1B68094A12881B79FF2B00D008BD062AFC
S3150800877CFCD10121002000F0EDF8FFF71BFFF5E70F
S3150800878C7C330020843300207033002010B502F0AF
S3150800879CEDFAB0B900F0F3F83A4B1B68984209D3D6
S315080087AC03F5FA73374A13600024002C36D00024DC
S315080087BC002C4AD000F0E3F8334B1B68984259D288
S315080087CC10BD324A1080324B9C894FF4006002F07F
S315080087DC6FFE844213D02E4B9C8940F6060002F09D
S315080087EC67FE8442D6D103F0B5FD284B1B88002BB7
S315080087FCD0D002F0E5FA254B00221A80CAE70120F0
S3150800880C02F090FE214B1B88002BC3D003F012FEFE
S3150800881C02F0D6FA1D4B00221A80BBE7C4EB0412F1
S3150800882C53001C4A13441C4A1360022002F07AFEB9
S3150800883C164B1B880BB90134B7E703F0FBFD02F0A6
S3150800884CBFFA124B00221A80F5E7144B03EB84137C
S3150800885C134A1360052002F065FE0C4B1B880BB9F6
S3150800886C0134A5E703F0E6FD02F0AAFA074B00224D
S3150800887C1A80F5E742F210721A44034B1A6003F099
S3150800888C35FD9DE744010020380100207033002097
S3150800889CBC3300208C33002088330020003A00209B
S315080088AC803300200B4B1B68C3F3072050FA83F266
S315080088BCC3F30740104400EB1360002305E0054A98
S315080088CC1A441279104480B20133372BF7D9404237
S315080088DC80B270470000002008B5FFF7E3FF044B91
S315080088EC9B8F984201D0002008BD0120FCE700BFF1
S315080088FC0000002008B5054B1A68054B9A4201D0B2
S3150800890C002008BDFFF7E8FFFBE700BF00000020CA
S3150800891CA2E742CE08B5FFF7C5FF014B988708BDFD
S3150800892C0000002008B5FFF7E5FF68B9074B084AB1
S3150800893C1A60002304E0054A1A4400211171013318
S3150800894C372BF8D9FFF7E6FF08BD00BF000000205B
S3150800895CA2E742CE70B505460E46FFF7CBFF044696
S3150800896C10B1372D02D90024204670BD024B1D4488
S3150800897C2E71FFF7CFFFF7E700000020704708B508
S3150800898C00F01EFA08BD0000014A024B9A607047B7
S3150800899C0080000800ED00E030B58DB00024079487
S315080089AC089409940A940B94244B1A6B42F080028F
S315080089BC1A631A6B02F080020192019A1A6B42F042
S315080089CC04021A631A6B02F004020292029A1A6BD8
S315080089DC42F001021A631A6B02F001020392039A1F
S315080089EC1A6B42F002021A631A6B02F00202049224
S315080089FC049A1A6B42F008021A631A6B02F0080200
S31508008A0C0592059A1A6B42F040021A631B6B03F027
S31508008A1C40030693069B0A4D22468021284600F001
S31508008A2C2FFF802307930123089309940A9407A917
S31508008A3C284600F037FE0DB030BD00BF00380240A6
S31508008A4C0004024030B5B9B0342200212BA803F03B
S31508008A5CEDFD002426942794289429942A94902290
S31508008A6C214602A803F0E2FD204B1A6C42F0805214
S31508008A7C1A641B6C03F080530093009B1C4B1A68FA
S31508008A8C42F440421A601B6803F440430193019B6D
S31508008A9C01232B934FF4A0232C93022531954FF4E5
S31508008AAC80033293082333934FF4D8733493359554
S31508008ABC36952BA800F028FF00F0E8FE0F23269326
S31508008ACC279528944FF4A05329934FF480532A934F
S31508008ADC072126A801F0A6F94FF480730293159482
S31508008AEC02A801F079FA39B030BD00BF003802404F
S31508008AFC0070004008B5FFF747FF00F049F9FFF78B
S31508008B0CA1FFFFF749FFFFF713FDFFF721FDFCE770
S31508008B1C82B00A4B1A6C42F080521A641A6C02F034
S31508008B2C80520092009A5A6C42F480425A645B6CEA
S31508008B3C03F480430193019B02B07047003802404E
S31508008B4CF0B58DB000230793089309930A930B93FA
S31508008B5C02683A4B9A4201D00DB0F0BDA3F590438A
S31508008B6C1A6B42F000721A631A6B02F000720092CA
S31508008B7C009A1A6B42F080621A631A6B02F08062D2
S31508008B8C0192019A1A6B42F000621A631A6B02F090
S31508008B9C00620292029A1A6B42F004021A631A6B6A
S31508008BAC02F004020392039A1A6B42F001021A634A
S31508008BBC1A6B02F001020492049A1A6B42F0020232
S31508008BCC1A631A6B02F002020592059A1A6B42F0A6
S31508008BDC40021A631B6B03F040030693069B322371
S31508008BEC07930226089603250A950B240B9407A9C6
S31508008BFC134800F057FD8623079308960027099714
S31508008C0C0A950B9407A90F4800F04CFD4FF4005336
S31508008C1C0793089609970A950B9407A90A4800F032
S31508008C2C41FD4FF420530793089609970A950B9420
S31508008C3C07A9064800F036FD8EE700BF0080024003
S31508008C4C00080240000002400004024000180240DE
S31508008C5C00B589B0002303930493059306930793F1
S31508008C6C0268144B9A4202D009B05DF804FB03F56E
S31508008C7CF8331A6C42F480221A641A6C02F48022B5
S31508008C8C0192019A1A6B42F008021A631B6B03F0E5
S31508008C9C08030293029B4FF4407303930223049335
S31508008CAC032306930723079303A9034800F0FAFC4A
S31508008CBCDAE700BF00480040000C02407047FEE7A8
S31508008CCCFEE7FEE7FEE770477047704708B500F009
S31508008CDC6BF808BD054BD3F8882042F47002C3F82C
S31508008CEC88204FF000629A60704700BF00ED00E0E4
S31508008CFCDFF834D0002103E00C4B5B5843500431A9
S31508008D0C0B480C4B42189A42F6D30B4A02E0002346
S31508008D1C42F8043B094B9A42F9D3FFF7DBFF03F001
S31508008D2C47FCFFF7E7FE70470000082098C60008C6
S31508008D3C400000204C0000204C000020403A002047
S31508008D4CFEE7000010B504460E4B18784FF47A73FC
S31508008D5CB3FBF0F30C4A1068B0FBF3F000F08EF896
S31508008D6C68B90F2C01D901200AE0002221464FF0E0
S31508008D7CFF3000F051F8054B1C60002000E0012084
S31508008D8C10BD00BF44000020400000204800002011
S31508008D9C08B5032000F02EF80020FFF7D3FFFFF7E5
S31508008DACB7FE002008BD0000034A1168034B1B7868
S31508008DBC0B441360704700BFCC020020440000200F
S31508008DCC014B1868704700BFCC02002038B5044622
S31508008DDCFFF7F6FF0546B4F1FF3F02D0044B1B78AC
S31508008DEC1C44FFF7EDFF401BA042FAD338BD00BF69
S31508008DFC440000200649CB6823F4E0631B041B0CD3
S31508008E0C000200F4E0600343024A1A43CA60704742
S31508008E1C00ED00E00000FA0530B4154BDB68C3F32F
S31508008E2C0223C3F10704042C28BF04241D1D062D98
S31508008E3C14D9033B4FF0FF3505FA04F421EA040173
S31508008E4C994005FA03F322EA03031943002807DBC2
S31508008E5C0901C9B2074B195430BC70470023E9E71E
S31508008E6C00F00F000901C9B2034B1954F4E700BF0F
S31508008E7C00ED00E000E400E014ED00E00138B0F18C
S31508008E8C807F0AD2064B5860064AF02182F82310D6
S31508008E9C0020986007221A6070470120704700BFAF
S31508008EAC10E000E000ED00E05079137943EA002366
S31508008EBC07480B50D07893781B0443EA0063507824
S31508008ECC43EA002312781343024A8B50704700BFBB
S31508008EDC4080024044800240016841F218028B58D7
S31508008EEC43F400538B507047016841F218028B58B3
S31508008EFC43F002038B50704770B59EB0044629B1F7
S31508008F0C4FF40063C3604FF480438360E369002B1E
S31508008F1C68D14FF48063079321680B68374A1A4067
S31508008F2CA368E06803430798034343F400731343A9
S31508008F3C0B6023681D680120FFF748FF23681D6036
S31508008F4C236840225A6023685D680120FFF73EFFBC
S31508008F5C23685D60236800259D602368DD602268B0
S31508008F6C936923F0BE031B041B0C43F08003936127
S31508008F7C23689E690120FFF729FF23689E612368F1
S31508008F8CDD612368DD690120FFF720FF2368DD61B9
S31508008F9C216841F218054B59194A1A40194B1343C3
S31508008FAC4B5123685E590120FFF710FF23685E5169
S31508008FBC236803F58053144A1A60236803F5805313
S31508008FCC1D680120FFF702FF236803F580531D6017
S31508008FDCA369012B09D0626900212046FFF764FFBB
S31508008FEC1EB070BD0023079396E7216841F21C0258
S31508008FFC8858064B03438B50EDE700BF0F8120FFC3
S3150800900C233FDEF8040020028020C1024000010044
S3150800901C10B582B00446002301930268136843F026
S3150800902C0803136003681B6801930120FFF7CEFE43
S3150800903C2368019A1A6002B010BD10B582B00446B6
S3150800904C002301930268136843F004031360036852
S3150800905C1B6801930120FFF7B9FE2368019A1A6071
S3150800906C02B010BD30B583B00546002301930268E3
S3150800907C41F21804135943F48013135103681B590E
S3150800908C01930120FFF7A2FE2B68019A1A5103B02F
S3150800909C30BDF0B490F84540012C31D0012480F84D
S315080090AC4540022480F84440C162002401E0F9607E
S315080090BC01349C4217D265014F194FF480164E5154
S315080090CC40F2F45606FB0426BE60C6691EB94E5914
S315080090DC46F440064E515D1EA542E8D9651C01EBC7
S315080090EC4515FD60E4E7026841F21003D1500123EF
S315080090FC80F84430002380F845301846F0BC704799
S3150800910C0220FBE7F0B490F84540012C2ED0012440
S3150800911C80F84540022480F844408162002401E02E
S3150800912CE96001349C4214D266018D194FF0004750
S3150800913C8F5144F2F4566E6040F2F45606FB042640
S3150800914CAE605E1EA642EBD9661C01EB4616EE60B7
S3150800915CE7E7026841F20C03D150012380F844304A
S3150800916C002380F845301846F0BC70470220FBE710
S3150800917C90F84530012B00F08580012380F84530A6
S3150800918C022380F84430B1B1C36A1A68002A1ADB84
S3150800919C30B440F2F45291421DD93B4AA2FB01422B
S315080091AC920A40F2F45404FB121404B10132012A57
S315080091BC11D0002347E0012380F84430002280F8C0
S315080091CC452018467047122380F84430002380F84F
S315080091DC4530012070471A6842F040521A60C36A3B
S315080091ECC1F30C015960C26A136843F0004313605B
S315080091FCC36ADB68C362036841F214029A5812F018
S3150800920C040F08D041F2140204219950026841F265
S3150800921C04030021D150012380F84430002380F840
S3150800922C4530184630BC7047C56A2C6844F08054E3
S3150800923C2C6011E0C56A2C6844F000442C60C46AA2
S3150800924CE468C46201339A42D5D9C56A2C6824F0FD
S3150800925C40542C60002BE7D0C46A40F2F455656084
S3150800926C541E9C42E6D1C56A2C6844F000542C6006
S3150800927C064C04FB021404F2F454C56AC4F30C0439
S3150800928C6C60D7E7022070470BB002AC0CFAFFFFF4
S3150800929C90F84530012B40D0012380F84530022345
S315080092AC80F84430836A1A68002A28DB1A6812F494
S315080092BC807F19D0826B01328263012A12D04363F4
S315080092CC1A68C2F30D42043AC263026B92680264CE
S315080092DCDB688362012380F84430002380F845302C
S315080092EC184670470363EAE71A6812F4007F0ED033
S315080092FC03630022426301228263DB6883620123D3
S3150800930C80F84430002280F8452018467047826B56
S3150800931C01328263DB688362F1E702207047F8B595
S3150800932C90F84430DBB2822B33D01646054682239E
S3150800933C80F844300268136903F01C03048AE402BB
S3150800934CA4B223438C0104F4F8641C4344F00104CE
S3150800935C1461FFF735FD074614F0010F10D0FFF71F
S3150800936C2FFDC01BB0F5803F02D22B681C69F3E7B2
S3150800937C012385F84430002385F84530032007E09F
S3150800938C2B685B699BB23360012385F84430002057
S3150800939CF8BD0220FCE790F84430DBB2422B32D001
S315080093AC70B50546422380F844300068036903F01B
S315080093BC1C032C8AE402A4B223438C0104F4F8643B
S315080093CC1C4344F0030492B242612B681C61FFF7FC
S315080093DCF7FC064614F0010F10D0FFF7F1FC801BC2
S315080093ECB0F5803F02D22B681C69F3E7012385F898
S315080093FC4430002385F84530032003E0012385F823
S3150800940C4430002070BD02207047000070B582B051
S3150800941C00230193002800F00C81044690F8443090
S3150800942C002B32D0844B5A6C42F480425A645B6CE3
S3150800943C03F480430093009B804B5A6822F4000285
S3150800944C5A605A68216A0A435A60236803F580539E
S3150800945C1A6842F001021A60FFF7B2FC0546236847
S3150800946C03F58052126812F0010F13D0FFF7A8FC0F
S3150800947C401BB0F5FA7FF2D9032584F84450002333
S3150800948C84F84530284602B070BD80F84530FFF7A1
S3150800949C57FBC7E71D6925F01C0500F077FD684BDF
S315080094AC0344684A934255D845F0080523681D615C
S315080094BC4FF4004200212046FFF76DFF05460028B1
S315080094CC60D1FF20FFF782FC6368002B00F09180C7
S315080094DCFFF776FC064601AA01212046FFF71FFF77
S315080094ECFFF76EFC801B41F28833984252D8019BD9
S315080094FC13F0040FEFD04FF4805200212046FFF7EB
S3150800950C4AFF002852D1FFF75BFC064601AA012147
S3150800951C2046FFF704FFFFF753FC801B41F2883304
S3150800952C98424BD8019B13F0200FEFD001AA1F21AC
S3150800953C2046FFF7F4FE00284CD1019B13F0100FC0
S3150800954C50D04FF40062E26013F0040F4DD00023A4
S3150800955CA3605EE03C4B03443C4A934202D845F078
S3150800956C0C05A3E73A4B03443A4A93429ED93A4B25
S3150800957C03443A4A934202D845F0040596E745F067
S3150800958C100593E701212046FFF7B6FC012584F860
S3150800959C445077E701212046FFF7AEFC012384F8F7
S315080095AC4430002384F8453003256BE70121204617
S315080095BCFFF7A2FC012584F8445063E701212046F5
S315080095CCFFF79AFC012384F84430002384F84530CD
S315080095DC032557E701212046FFF78EFC012584F861
S315080095EC44504FE70022E260AEE74FF48043A36095
S315080095FC0FE0E268C2F3CF02A368C3F34F031A4322
S3150800960C00212046FFF7C7FE58B940F6FF70FFF752
S3150800961CDDFB00212046FFF76FFC012384F844305C
S3150800962C30E701212046FFF767FC012584F84450F2
S3150800963C28E7012526E700BF00380240003801401C
S3150800964C00D3CEFEBFE1E40040F1E9FD3F787D0191
S3150800965C00796CFCFF596202001F0AFA7FF0FA02C5
S3150800966C38B590F84530012B1AD00446012580F8F8
S3150800967C4550022380F84430FFF7CAFC2046FFF712
S3150800968CDCFC2046FFF7EEFC2046FFF725FC2046BF
S3150800969CFFF72AFC84F84450002084F8450038BDAE
S315080096AC0220FCE700230F2B00F2E180F0B583B013
S315080096BC39E0092200E00022B2403A4302346C4EEB
S315080096CC46F824206B4A1468EA4302EA04064F68F3
S315080096DC17F4803F01D045EA0406664C2660646898
S315080096EC02EA04064F6817F4003F01D045EA04065F
S315080096FC604C6660A46802EA04064F6817F4801F7B
S3150800970C01D045EA04065B4CA660E46822404E6824
S3150800971C16F4001F01D045EA0402564CE2600133E8
S3150800972C0F2B00F2A28001229A400C6804EA02056B
S3150800973CAA42F4D14C68661E112C18BF012E01D909
S3150800974C122C12D186685F000324BC4026EA040654
S3150800975CCC68BC4034438460466826EA02064C68EA
S3150800976CC4F300129A4032434260C2685F00032673
S3150800977CBE40F64332408C68BC401443C4604A6809
S3150800978C122A18BF022A13D1DC08083450F824E030
S3150800979C03F007024FEA820C0F2202FA0CF22EEAA9
S315080097AC020E0A6902FA0CF242EA0E0240F824206A
S315080097BC026816404A6802F00302BA403243026055
S315080097CC4A6812F0805FAAD02B4A546C44F4804441
S315080097DC5464526C02F480420192019A9C08A61CAD
S315080097EC234A52F8267003F0030296000F22B24061
S315080097FC27EA0207214A90423FF45DAF02F58062E0
S3150800980C904222D002F58062904220D002F5806206
S3150800981C90421ED002F5806290421CD002F58062FE
S3150800982C90421AD002F58062904218D002F58062F6
S3150800983C904216D002F58062904214D002F58062EE
S3150800984C90423FF436AF0A2236E7012234E7022269
S3150800985C32E7032230E704222EE705222CE70622FC
S3150800986C2AE7072228E7082226E703B0F0BD704747
S3150800987C00380140003C014000380240000002401C
S3150800988C12B90904816170478161704710B582B0BD
S3150800989C1B4B1A6C42F080521A641B6C03F08053F3
S315080098AC0193019B174A136843F480331360FFF73F
S315080098BC87FA0446134B5B6813F4803F08D1FFF70D
S315080098CC7FFA001BB0F57A7FF4D9032002B010BDDD
S315080098DC0C4A136843F400331360FFF771FA044615
S315080098EC084B5B6813F4003F07D1FFF769FA001BB6
S315080098FCB0F57A7FF4D90320E8E70020E6E700BF45
S3150800990C0038024000700040002800F0128270B542
S3150800991C82B00446036813F0010F29D0A24B9B684A
S3150800992C03F00C03042B1AD09F4B9B6803F00C0313
S3150800993C082B0FD06368B3F5803F40D0002B54D169
S3150800994C994B1A6822F480321A601A6822F480221B
S3150800995C1A6039E0944B5B6813F4800FEAD0924B8B
S3150800996C1B6813F4003F03D06368002B00F0E381F7
S3150800997C236813F0020F75D08B4B9B6813F00C0FF2
S3150800998C5ED0894B9B6803F00C03082B53D0E36815
S3150800999C002B00F08A80844A136843F00103136095
S315080099ACFFF70EFA0546804B1B6813F0020F73D1AE
S315080099BCFFF706FA401B0228F5D90320BEE17A4ABE
S315080099CC136843F48033136063682BB3FFF7F8F915
S315080099DC0546754B1B6813F4003FC9D1FFF7F0F920
S315080099EC401B6428F5D90320A8E1B3F5A02F09D0AC
S315080099FC6D4B1A6822F480321A601A6822F4802297
S31508009A0C1A60E1E7684B1A6842F480221A601A68F1
S31508009A1C42F480321A60D7E7FFF7D2F90546624B53
S31508009A2C1B6813F4003FA3D0FFF7CAF9401B642840
S31508009A3CF5D9032082E15C4B5B6813F4800FA6D141
S31508009A4C594B1B6813F0020F04D0E368012B01D0A5
S31508009A5C012073E1544A136823F0F803216943EA99
S31508009A6CC1031360236813F0080F46D0636983B3E8
S31508009A7C4D4A536F43F001035367FFF7A1F90546A7
S31508009A8C494B5B6F13F0020F37D1FFF799F9401B5F
S31508009A9C0228F5D9032051E1434A136823F0F80349
S31508009AAC216943EAC1031360DCE73F4A136823F0D4
S31508009ABC01031360FFF784F905463B4B1B6813F04B
S31508009ACC020FCFD0FFF77CF9401B0228F5D90320EB
S31508009ADC34E1354A536F23F001035367FFF770F9E6
S31508009AEC0546314B5B6F13F0020F06D0FFF768F98A
S31508009AFC401B0228F5D9032020E1236813F0040F34
S31508009B0C7ED0294B1B6C13F0805F1ED1264B1A6C2A
S31508009B1C42F080521A641B6C03F080530193019B2C
S31508009B2C0125224B1B6813F4807F10D0A368012BE8
S31508009B3C21D0002B3CD11C4B1A6F22F001021A675C
S31508009B4C1A6F22F004021A671AE00025E9E7174A89
S31508009B5C136843F480731360FFF732F90646134B08
S31508009B6C1B6813F4807FE1D1FFF72AF9801B642860
S31508009B7CF5D90320E2E00C4A136F43F0010313678F
S31508009B8CA3685BB3FFF71CF90646074B1B6F13F06C
S31508009B9C020F34D1FFF714F9801B41F2883398422F
S31508009BACF3D90320CAE000BF003802400070004019
S31508009BBC052B09D0644B1A6F22F001021A671A6F2B
S31508009BCC22F004021A67DBE75F4B1A6F42F00402B5
S31508009BDC1A671A6F42F001021A67D1E7FFF7F0F815
S31508009BEC0646594B1B6F13F0020F08D0FFF7E8F81F
S31508009BFC801B41F288339842F3D903209EE0FDB9C5
S31508009C0CA369002B00F099804F4A926802F00C0267
S31508009C1C082A59D0022B19D04B4A136823F08073A3
S31508009C2C1360FFF7CDF80446474B1B6813F0007F0B
S31508009C3C48D0FFF7C5F8001B0228F5D903207DE0AC
S31508009C4C414A136C23F080531364D9E73E4A1368D0
S31508009C5C23F080731360FFF7B3F805463A4B1B687D
S31508009C6C13F0007F06D0FFF7ABF8401B0228F5D996
S31508009C7C032063E0E369226A1343626A43EA8213A8
S31508009C8CA26A5208013A43EA0243E26A43EA0263C9
S31508009C9C226B43EA02732C4A5360136843F08073B1
S31508009CAC1360FFF78DF80446274B1B6813F0007FEB
S31508009CBC06D1FFF785F8001B0228F5D903203DE0ED
S31508009CCC00203BE0002039E01F4A5268012B37D0B0
S31508009CDC02F48003E1698B4201D001202EE002F0E8
S31508009CEC3F03216A8B4201D0012027E0616A47F6BF
S31508009CFCC0731340B3EB811F01D001201EE002F4A0
S31508009D0C4031A36A5B08013BB1EB034F01D001203C
S31508009D1C14E002F07063E16AB3EB016F01D0012025
S31508009D2C0CE002F0E042236BB2EB037F0AD0012071
S31508009D3C04E001207047012000E0002002B070BD4D
S31508009D4C0120FBE70020F9E700380240324B9B68FC
S31508009D5C03F00C03042B5CD0082B01D02F4870475A
S31508009D6C2DE9F04B2C4B5A6802F03F025B6813F452
S31508009D7C800F2BD0284B5B68C3F388131E4600272D
S31508009D8C5C010025E41A65EB0705A90141EA946113
S31508009D9CA001001B61EB0501CB0043EA5073C4001C
S31508009DACA01943EB07014B0243EAD0534402204661
S31508009DBC19460023FEF73CFA174B5B68C3F30143BD
S31508009DCC01335B00B0FBF3F0BDE8F08B124B5B681C
S31508009DDCC3F388131E4600275C010025E41A65EBBD
S31508009DEC0705A90141EA9461A001001B61EB050175
S31508009DFCCB0043EA5073C400A01943EB07018B024E
S31508009E0C43EA90538402204619460023FEF710FABB
S31508009E1CD2E70348704700BF003802400024F4001C
S31508009E2C00127A00002800F0A38070B50446524B45
S31508009E3C1B6803F00F038B420CD24F4A136823F0AE
S31508009E4C0F030B431360136803F00F038B4201D007
S31508009E5C012070BD236813F0020F17D013F0040FFE
S31508009E6C04D0464A936843F4E0539360236813F08E
S31508009E7C080F04D0414A936843F4604393603F4A01
S31508009E8C936823F0F003A068034393600D46236898
S31508009E9C13F0010F31D06368012B20D0022B25D08B
S31508009EAC364A126812F0020F64D034498A6822F0D6
S31508009EBC030213438B60FEF783FF06462F4B9B6802
S31508009ECC03F00C036268B3EB820F16D0FEF778FF2B
S31508009EDC801B41F288339842F0D90320B9E7274A08
S31508009EEC126812F4003FE0D10120B2E7234A126847
S31508009EFC12F0007FD9D10120ABE71F4B1B6803F08A
S31508009F0C0F03AB420CD91C4A136823F00F032B43DF
S31508009F1C1360136803F00F03AB4201D0012098E7D6
S31508009F2C236813F0040F06D0144A936823F4E053FD
S31508009F3CE1680B439360236813F0080F07D00F4AA8
S31508009F4C936823F46043216943EAC1039360FFF7DE
S31508009F5CFDFE0A4B9B68C3F30313094AD35CD8402E
S31508009F6C084B1860084B1868FEF7ECFE002070E7E3
S31508009F7C0120704701206CE7003C02400038024083
S31508009F8C60C600084000002048000020014B1868F5
S31508009F9C704700BF4000002008B5FFF7F7FF044BD9
S31508009FAC9B68C3F38223034AD35CD84008BD00BF21
S31508009FBC0038024070C6000808B5FFF7E7FF044BE7
S31508009FCC9B68C3F34233034AD35CD84008BD00BF31
S31508009FDC0038024070C60008F0B583B00446036822
S31508009FEC13F0010F0CD0B54B9A6822F400029A6054
S31508009FFC9A68416B0A439A60436BC3B1002600E02A
S3150800A00C0026236813F4002F15D0AC4AD2F88C30EE
S3150800A01C23F44013E16B0B43C2F88C30E36BB3F5B6
S3150800A02C801F06D0002B00F04581002504E0012690
S3150800A03CE7E70126F6E70025236813F4801F0FD0FF
S3150800A04C9E4AD2F88C3023F44003216C0B43C2F899
S3150800A05C8C30236CB3F5800F00F02E8103B90125E3
S3150800A06C236813F0807F00D0012613F0200F40F0F0
S3150800A07C2781236813F0100F0CD0904BD3F88C2043
S3150800A08C22F08072C3F88C20D3F88C20A16B0A437B
S3150800A09CC3F88C20236813F4804F08D0874AD2F86B
S3150800A0AC903023F44033616E0B43C2F8903023682A
S3150800A0BC13F4004F08D0814AD2F8903023F4402389
S3150800A0CCA16E0B43C2F89030236813F4803F08D076
S3150800A0DC7A4AD2F8903023F44013E16E0B43C2F857
S3150800A0EC9030236813F4003F08D0744AD2F89030A5
S3150800A0FC23F44003216F0B43C2F89030236813F006
S3150800A10C400F08D06D4AD2F8903023F00303616CE7
S3150800A11C0B43C2F89030236813F0800F08D0674AB7
S3150800A12CD2F8903023F00C03A16C0B43C2F8903094
S3150800A13C236813F4807F08D0604AD2F8903023F055
S3150800A14C3003E16C0B43C2F89030236813F4007F9C
S3150800A15C08D05A4AD2F8903023F0C003216D0B432D
S3150800A16CC2F89030236813F4806F08D0534AD2F89B
S3150800A17C903023F44073616D0B43C2F8903023681A
S3150800A18C13F4006F08D04D4AD2F8903023F440638C
S3150800A19CA16D0B43C2F89030236813F4805F08D086
S3150800A1AC464AD2F8903023F44053E16D0B43C2F87B
S3150800A1BC9030236813F4005F08D0404AD2F89030E8
S3150800A1CC23F44043216E0B43C2F89030236813F4F2
S3150800A1DC800F08D0394AD2F8903023F08063A16FEB
S3150800A1EC0B43C2F89030236813F4001F0DD0334A82
S3150800A1FCD2F8903023F00063E16F0B43C2F890302D
S3150800A20CE36FB3F1006F00F0C180236813F0080FF9
S3150800A21C00D0012513F4802F08D0284AD2F89030A4
S3150800A22C23F04073616F0B43C2F89030236813F424
S3150800A23C000F09D0214AD2F8903023F08053D4F875
S3150800A24C80100B43C2F89030236813F0806F09D046
S3150800A25C1A4AD2F8903023F00053D4F884100B43E2
S3150800A26CC2F89030236813F0006F09D0134AD2F85D
S3150800A27C8C3023F00073D4F888100B43C2F88C305A
S3150800A28C236813F0805F09D00C4AD2F88C3023F07F
S3150800A29C8063D4F88C100B43C2F88C30002E77D11F
S3150800A2AC2368B3F1007F73D0002D40F004810020A1
S3150800A2BC03B0F0BD0125BFE60126CFE60038024003
S3150800A2CCB74B1A6C42F080521A641B6C03F080531D
S3150800A2DC0193019BB34A136843F480731360FEF72A
S3150800A2EC6FFD0746AF4B1B6813F4807F06D1FEF74C
S3150800A2FC67FDC01B6428F5D90320D9E7A84B1B6F4B
S3150800A30C13F4407315D0226B02F440729A4210D0A3
S3150800A31CA34B1A6F22F44072196F41F480311967F6
S3150800A32C196F21F4803119671A671B6F13F0010F27
S3150800A33C12D1236B03F44072B2F5407F1DD0984AB4
S3150800A34C936823F4F813936095490B6F226BC2F349
S3150800A35C0B0213430B678CE6FEF732FD0746904B50
S3150800A36C1B6F13F0020FE4D1FEF72AFDC01B41F256
S3150800A37C88339842F3D903209AE78948826822F4ED
S3150800A38CF812894919400A438260DDE701253CE742
S3150800A39C834A136823F080631360FEF711FD0646A3
S3150800A3AC7F4B1B6813F0006F06D0FEF709FD801B68
S3150800A3BC6428F5D903207BE7236813F0010F13D023
S3150800A3CC636B8BB9764AD2F88430D2F884106068FD
S3150800A3DC03F4403343EA801301F070610B43A16820
S3150800A3EC43EA0173C2F88430236813F4002F03D0B0
S3150800A3FCE26BB2F5801F06D013F4801F1ED0236CB7
S3150800A40CB3F5800F1AD1664AD2F88430D2F8841084
S3150800A41C606803F4403343EA8013E06843EA006358
S3150800A42C01F0E0410B43C2F88430D2F88C3023F0AB
S3150800A43C1F03616A01390B43C2F88C30236813F089
S3150800A44C807F11D0564AD2F88400D2F884106668F8
S3150800A45C23691B0443EA861300F07060034301F07A
S3150800A46CE0410B43C2F88430236813F0007F0DD00B
S3150800A47C626823691B0443EA8213E26843EA0263AF
S3150800A48CA26843EA0273464AC2F88430444A1368FF
S3150800A49C43F080631360FEF793FC0646404B1B683B
S3150800A4AC13F0006F7FF400AFFEF78AFC801B64285C
S3150800A4BCF4D90320FCE63A4A136823F08053136058
S3150800A4CCFEF77EFC0546364B1B6813F0005F06D07C
S3150800A4DCFEF776FC401B6428F5D90320E8E62368CA
S3150800A4EC13F4002F01D0E26B22B113F4801F1DD098
S3150800A4FC236CDBB92A4AD2F88830D2F888106069FE
S3150800A50C03F4403343EA8013A06943EA006301F07D
S3150800A51CE0410B43C2F88830D2F88C3023F4F85358
S3150800A52CA16A013943EA0123C2F88C30236813F473
S3150800A53C001F03D0E36FB3F1006F37D0236813F015
S3150800A54C080F19D0164AD2F88810D2F888306069E4
S3150800A55C03F4403343EA801301F070610B43E1695D
S3150800A56C43EA0173C2F88830D2F88C3023F44033AE
S3150800A57CE16A0B43C2F88C30094A136843F08053DE
S3150800A58C1360FEF71DFC0446054B1B6813F0005FB1
S3150800A59C1FD1FEF715FC001B6428F5D9032087E6A6
S3150800A5AC0038024000700040FFFCFF0F0A4AD2F840
S3150800A5BC8800D2F888106569236A1B0443EA851358
S3150800A5CC00F07060034301F0E0410B43C2F8883099
S3150800A5DCB4E700206CE600BF0038024010B504460C
S3150800A5EC83680269134342691343C26913430168BA
S3150800A5FC0868994A024013430B602268536823F48F
S3150800A60C4053E1680B435360A269236A1A432168D5
S3150800A61C8B6823F4306313438B6023688F4A934209
S3150800A62C18D08F4A934228D08E4A93423DD08E4AF0
S3150800A63C934250D08D4A934262D08D4A934277D03A
S3150800A64C8C4A934200F08C808B4A934200F0A0808F
S3150800A65C1023B6E0894BD3F8903003F00303032B91
S3150800A66C09D8DFE803F00204AD060123A9E00423A8
S3150800A67CA7E00823A5E01023A3E0804BD3F890307D
S3150800A68C03F00C030C2B0ED8DFE803F0070D0D0DA9
S3150800A69C090D0D0DA90D0D0D0B00002391E00423DA
S3150800A6AC8FE008238DE010238BE0744BD3F89030A1
S3150800A6BC03F03003102B0AD006D9202B00F091801A
S3150800A6CC302B06D108237CE01BB9002379E0042340
S3150800A6DC77E0102375E0694BD3F8903003F0C0038C
S3150800A6EC402B09D005D9802B7DD0C02B06D1082349
S3150800A6FC67E01BB9002364E0042362E0102360E0E2
S3150800A70C5E4BD3F8903003F44073B3F5807F0BD0CF
S3150800A71C07D9B3F5007F68D0B3F5407F06D1082377
S3150800A72C4FE01BB900234CE004234AE0102348E011
S3150800A73C524BD3F8903003F44063B3F5806F0BD0CB
S3150800A74C07D9B3F5006F52D0B3F5406F06D108237D
S3150800A75C37E01BB9012334E0042332E0102330E040
S3150800A76C464BD3F8903003F44053B3F5805F0BD0C7
S3150800A77C07D9B3F5005F3CD0B3F5405F06D1082383
S3150800A78C1FE01BB900231CE004231AE0102318E071
S3150800A79C3A4BD3F8903003F44043B3F5804F0BD0C3
S3150800A7AC07D9B3F5004F26D0B3F5404F06D1082389
S3150800A7BC07E01BB9002304E0042302E0102300E0A1
S3150800A7CC0223E269B2F5004F17D0082B00F2B380CA
S3150800A7DCDFE803F0768B95B19EB1B1B1A8000223E0
S3150800A7ECEFE70223EDE70223EBE70223E9E702236F
S3150800A7FCE7E70223E5E70223E3E7082B5DD8DFE862
S3150800A80C03F0051F3F5C485C5C5C5300FFF7C4FB18
S3150800A81C6268530803EB4003B3FBF2F39BB20020C8
S3150800A82CA3F110014FF6EF72914200F287809AB2AB
S3150800A83C22F00F02C3F3420313432268D36050E09D
S3150800A84CFFF7BAFB6268530803EB4003B3FBF2F35A
S3150800A85C9BB20020E4E700BFF369FFEF001001404C
S3150800A86C0044004000480040004C004000500040A6
S3150800A87C0014014000780040007C0040003802407B
S3150800A88C6268304B03EB5203B3FBF2F39BB2002026
S3150800A89CC6E7FFF75BFA6268530803EB4003B3FBA2
S3150800A8ACF2F39BB20020BBE76268530803F58033CA
S3150800A8BCB3FBF2F39BB20020B2E701200023AFE70B
S3150800A8CCFFF76AFB626800EB5203B3FBF2F39BB229
S3150800A8DC0020A3F110014FF6EF72914230D822688E
S3150800A8ECD36000232366636610BDFFF765FB6268B9
S3150800A8FC00EB5203B3FBF2F39BB20020E9E7626864
S3150800A90C114B03EB5203B3FBF2F39BB20020E0E7C7
S3150800A91CFFF71CFA626800EB5203B3FBF2F39BB227
S3150800A92C0020D6E76268530803F50043B3FBF2F33D
S3150800A93C9BB20020CDE701200023CAE70120D0E70F
S3150800A94C0120CEE70048E8010024F400436A13F01E
S3150800A95C010F06D00268536823F40033816A0B434F
S3150800A96C5360436A13F0020F06D00268536823F447
S3150800A97C8033C16A0B435360436A13F0040F06D045
S3150800A98C0268536823F48023016B0B435360436AB4
S3150800A99C13F0080F06D00268536823F40043416B82
S3150800A9AC0B435360436A13F0100F06D00268936882
S3150800A9BC23F48053816B0B439360436A13F0200F87
S3150800A9CC06D00268936823F40053C16B0B4393605B
S3150800A9DC436A13F0400F0AD00268536823F48013B5
S3150800A9EC016C0B435360036CB3F5801F0BD0436AA1
S3150800A9FC13F0800F06D00268536823F40023816C89
S3150800AA0C0B43536070470268536823F4C003416CC8
S3150800AA1C0B435360EBE72DE9F04104460F46164607
S3150800AA2C9846069D2368DB6937EA03030CBF0123A6
S3150800AA3C0023B3423AD1B5F1FF3FF3D0FEF7C0F984
S3150800AA4CA0EB0800A8421FD8F5B123681A6812F0C3
S3150800AA5C040FE7D0DA6912F4006FE3D04FF4006202
S3150800AA6C1A622268136823F4D073136022689368F9
S3150800AA7C23F00103936020236367A367E36700232E
S3150800AA8C84F87030032012E02268136823F4D0731C
S3150800AA9C13602268936823F001039360202363678D
S3150800AAACA367002384F87030032000E00020BDE87B
S3150800AABCF0812DE9F04383B01E46836F202B7FD19E
S3150800AACC04460D469046B2FA82F35B09002908BF84
S3150800AADC0123002B78D190F87030012B76D0012306
S3150800AAEC80F870300023C36722238367FEF768F962
S3150800AAFC0746A4F85880A4F85A80A368B3F5805F73
S3150800AB0C06D0A3B9226972B9FF22A4F85C2014E016
S3150800AB1C226922B940F2FF12A4F85C200DE0FF224C
S3150800AB2CA4F85C2009E07F22A4F85C2005E0B3F1C8
S3150800AB3C805F0DD00022A4F85C20B4F85C80B3F5D5
S3150800AB4C805F0FD04FF00009002384F870301DE0A9
S3150800AB5C22691AB97F22A4F85C20EEE73F22A4F8F2
S3150800AB6C5C20EAE7236913B14FF00009ECE7A94624
S3150800AB7C0025E9E723685B6A08EA030329F8023B20
S3150800AB8CB4F85A30013B9BB2A4F85A30B4F85A3090
S3150800AB9C9BB28BB100963B46002220212046FFF73C
S3150800ABAC3AFFA8B9002DE5D023685A6A5FFA88F3EC
S3150800ABBC134005F8013BE3E72023A367002000E0D8
S3150800ABCC022003B0BDE8F0830120FAE70220F8E77B
S3150800ABDC0320F6E730B583B004460023C367FEF7B7
S3150800ABECEFF8054623681B6813F0080F0CD1236889
S3150800ABFC1B6813F0040F15D120236367A367002085
S3150800AC0C84F8700003B030BD6FF07E4300930346A2
S3150800AC1C00224FF400112046FFF7FDFE0028E6D06F
S3150800AC2C0320EFE76FF07E4300932B4600224FF488
S3150800AC3C80012046FFF7EFFE0028DDD00320E1E770
S3150800AC4C68B310B50446436F03B3242363672268BD
S3150800AC5C136823F0010313602046FFF7BFFC012895
S3150800AC6C13D0636ABBB92268536823F490435360C4
S3150800AC7C2268936823F02A0393602268136843F0CA
S3150800AC8C010313602046FFF7A5FF10BD80F870304E
S3150800AC9CFDF7DEFFD9E72046FFF758FEE3E701206C
S3150800ACAC704708B5FDF76BFE08BD000010B5164BCE
S3150800ACBC08221A7000225A70272199706921D970B6
S3150800ACCC5B21197145215971104C114921600121DB
S3150800ACDC616022826361A261E2614FF40003236220
S3150800ACEC2046FEF793FB04230A4A0B492046FEF737
S3150800ACFCD0F90423094A0A492046FEF703FA2046E6
S3150800AD0CFEF7AEFC10BD00BF4801002084020020EF
S3150800AD1C00800240A01B0020D00200205003002017
S3150800AD2C201B0020074A1178074B19705178597067
S3150800AD3C91789970D178D9701179197152795A71AB
S3150800AD4C704700BF4801002090010020064B1A7876
S3150800AD5C02705A7842709A788270DA78C2701A79C8
S3150800AD6C02715B79437170474801002038B5124867
S3150800AD7CFEF78EFA10B10024204638BD0E4DAC8F66
S3150800AD8C2246296C0D4801F046FC2A6B136843F0E1
S3150800AD9C004313600023AB632B6841F214029A58E4
S3150800ADAC12F0800FE8D041F214028021995041F23A
S3150800ADBC080200219950DFE784020020BC330020EA
S3150800ADCC38B5184BDC6AFDF7DAFD00F1FA0523688D
S3150800ADDC002B05DAFDF7D3FDA842F8D9012300E0CC
S3150800ADEC002383B10F4B1B6841F214029A5812F0D8
S3150800ADFC200F07D041F214022021995041F2040287
S3150800AE0C0021995038BD084B1D88064CE36A2A4622
S3150800AE1C0649986801F0FFFB29462046FEF7A8F973
S3150800AE2CE0E700BF8402002070330020BC3300200A
S3150800AE3C352303700123437081700330704700007B
S3150800AE4C3623037004234370024BDB69C0F80230C7
S3150800AE5C06307047500100203223037004234370D8
S3150800AE6C024B5B6AC0F8023006307047500100206E
S3150800AE7C372303700323437001228270C3700623A1
S3150800AE8C037105307047FF230370013070470000CB
S3150800AE9C0346014400208B4234D210B410E0362A03
S3150800AEAC23D0FF2A2BD0352A05D1987803E0D3F87E
S3150800AEBC0240154A94625A78023213448B421ED2C7
S3150800AECC1A78332A16D0EAD8032A04D0062A07D0C9
S3150800AEDC012AF0D1EBE7D3F802400B4A1463EAE7F0
S3150800AEECD3F80240084AD462E5E7D3F80240064A8A
S3150800AEFCD461E0E7D3F80240034A1462DBE75DF855
S3150800AF0C044B7047704700BF50010020074B828CDA
S3150800AF1C1A80C28C5A80064B028D1A80428D5A8032
S3150800AF2C044B028E1A80428E5A807047B833002022
S3150800AF3CB4330020B0330020F8B50446012303705F
S3150800AF4C4370184B9A6982700025C570164A1268A8
S3150800AF5C4260058180274781144A1268C2600561E0
S3150800AF6C456185619E69324659691C3001F053FB6F
S3150800AF7C06F118002044C6F110022946043001F0E7
S3150800AF8C55FB4022294604F12C0001F04FFB3A46AA
S3150800AF9C294604F16C0001F049FB054B1B68C4F803
S3150800AFACEC30F8BD500100207CC60008B8330020F0
S3150800AFBC78C6000838B50A4C25682846FFF7BCFF42
S3150800AFCC012105F1F000FFF733FFFFF751FFFFF7FB
S3150800AFDC5AFF2368C11A184601F0F4F838BD00BFA9
S3150800AFEC8433002038B50B4C25682846FFF7A4FF98
S3150800AFFC032105F1F000FFF71BFFFFF721FFFFF711
S3150800B00C2BFFFFF740FF2368C11A184601F0DAF840
S3150800B01C38BD00BF8433002010B5114B1C6823784B
S3150800B02C022B01D0002010BD04220E49A01801F0F5
S3150800B03CE3FA98B90C4B9A69596904F11C0001F0AA
S3150800B04CDBFA08B10020EEE72269074B5A62074B78
S3150800B05C198804F1F000FFF71BFFE4E70020E2E78C
S3150800B06C843300207CC60008500100207033002071
S3150800B07C10B582B00C4C6061A1610023A3704FF629
S3150800B08CFF73ADF80430ADF806304FF4864101A8CD
S3150800B09C01F048F8606010B14FF488438380024B86
S3150800B0AC00221A8002B010BD50010020024B00226B
S3150800B0BC1A805A80704700BFB833002038B5984BB1
S3150800B0CC1B88B3F5937F15D059D840F20F129342CB
S3150800B0DC00F09A80B3F5887F47D3B3F5887F00F0E4
S3150800B0EC978040F22512934240F015818C4B4FF411
S3150800B0FC93721A808B4B1B7813F0020F00F0CB80DF
S3150800B10C884B1B7813F0020F40F0CD80844B1B69DB
S3150800B11C42F21072934200F3CF80814A03F57A7398
S3150800B12C13619378032B40F0A9807D48FFF7EEFE58
S3150800B13C7B4D288C00F0BCF90404688C00F0B8F937
S3150800B14C204340084FF47A7404FB00F00028C0F240
S3150800B15CB7802861724C216904F1080001F014FAD1
S3150800B16C40F255132380032075E0002B40F0D38062
S3150800B17C6B4B01229A704FF47A721A615FE0B3F541
S3150800B18CAB7F3AD030D9B3F5B57F00F0A78040F243
S3150800B19C6B12934240F0BF80624B1B7813F0020F80
S3150800B1AC00F0A1805F4B1B7813F0020F40F0A380D0
S3150800B1BC5B4B1B6942F21072934200F3A880584A03
S3150800B1CC03F57A7313619378032B00F09C80FFF7D1
S3150800B1DC09FF534C216904F1080001F0D5F94FF425
S3150800B1ECB5732380032036E040F25512934240F0A3
S3150800B1FC92804B4B4FF4AB721A804B4801F0CBF94B
S3150800B20C002862D1002026E0454B4FF488721A803C
S3150800B21C444B1B7813F0020F1ED0424B1B7813F0CD
S3150800B22C020F20D13E4B1B694EF65F22934202DC7D
S3150800B23C5B003B4A13613A4B9B78022B1AD0FFF7FB
S3150800B24CB9FE374C216904F1080001F09DF940F26A
S3150800B25C0F132380032038BD334801F09CF90028CE
S3150800B26CDBD10020F7E7FFF7D7FE0228DAD12C4B03
S3150800B27C02229A702A4B4FF47A721A61FFF7B2FEC1
S3150800B28C274C216904F1080001F07EF940F22513D8
S3150800B29C23800320DFE7244801F07DF900287FF49A
S3150800B2AC2FAF0020D7E7FFF7B7FE05287FF42EAFA0
S3150800B2BC1B4B03229A7038E70020194B1880CAE7F3
S3150800B2CC174B6FF000421A6144E7154B02229A702D
S3150800B2DC4FF47A721A61FFF7E9FE78E7104B40F2E1
S3150800B2EC6B121A8058E7104801F055F900287FF4BC
S3150800B2FC59AF0020AFE7FFF78FFE05287FF458AF4C
S3150800B30C074B03229A700648FFF700FE10E7002049
S3150800B31C034B18809FE7024B00221A8002209AE7FB
S3150800B32C500100207C3300205801002008B5FFF797
S3150800B33CC5FE08BD10B4013A0A4400E00231914238
S3150800B34C0BD20C784B7803EB04239BB2184480B2CF
S3150800B35C8342F3D9013080B2F0E702D05DF8044B92
S3150800B36C70470B781B02184480B28342F6D9013019
S3150800B37C80B2F3E770B4C5780D44EDB2134CE570A2
S3150800B38C83780E0A3344DBB2A37042786270007875
S3150800B39C20709CB2A64206D90132D2B20B4C62700E
S3150800B3AC0AB901302070C9B28D420CDA0133DBB20E
S3150800B3BC064A93703BB953780133DBB2537013B911
S3150800B3CC13780133137070BC704700BF78330020B4
S3150800B3DC10B5094C2368014603F10800FFF7CAFFAC
S3150800B3EC2368064A117819725178597291789972AC
S3150800B3FCD278DA7210BD00BF88330020783300206B
S3150800B40C1A4B00221A7006E0194A002122F813106A
S3150800B41C0133164A1370154B1B78002BF4D0134BBB
S3150800B42C00221A7009E0C3EB03125100114A0A44B0
S3150800B43C0021517601330D4A13700C4B1B78002BE7
S3150800B44CF1D00D4B4FF480621A80084B00221A700B
S3150800B45C07E00A4A02EB8312002191800133034A62
S3150800B46C1370024B1B78002BF3D070478401002015
S3150800B47CAC3300208C3300208C010020003A0020CD
S3150800B48C094B00221A70084B1B7863B91946074AF0
S3150800B49C32F813201AB10133034A1370F3E7034B3E
S3150800B4AC23F811007047704784010020AC33002044
S3150800B4BC030A43EA002080B27047000008B514223C
S3150800B4CC05490020FFF736FF10B1FFF7F1FF08BD5D
S3150800B4DC4FF6FF70FBE700BFCA33002038B50D4D99
S3150800B4EC2B7C6C7C04EB0324A4B2143CA4B220443D
S3150800B4FC082205F11A0180B2FFF71CFF224605F156
S3150800B50C2201FFF717FF10B1FFF7D2FF38BD4FF630
S3150800B51CFF70FBE7BC33002008B50620FFF7DEFFFB
S3150800B52C08BD000070B5B24B1C68042800F0968163
S3150800B53CB04BB14A1360B14A1360032859D002289C
S3150800B54C00F0C880052800F07281AD4B9B7B452B1B
S3150800B55C54D1AB4A157C537C03EB0521A94A1288B6
S3150800B56C91424BDC8DB2A74B1D80A54B1B7D13F06E
S3150800B57C3F0F43D1A24B5B7D002B3FD1A24B1C88BE
S3150800B58C0CB95B884BB19E4BDB8B9C4236D19C4BE2
S3150800B59C1A8C9D4B5B889A4230D1FFF78FFF4FF67A
S3150800B5ACFF7398422AD1964BDB7D062B00F0E98176
S3150800B5BC112B00F09F81012B20D1914B93F822304F
S3150800B5CC082B1BD18E4B002283F822209B8C4FF61E
S3150800B5DCF672934240F28A810933894A9384884BDE
S3150800B5EC5A8BDA839A8B1A845C83874A52889A8395
S3150800B5FC78E1637E03F00F03032B05D00023814A01
S3150800B60C1380824A137070BD238A002BF6D17F4BA8
S3150800B61C08221A70FDF79AF87C4B1B7813F0200F4A
S3150800B62C00F0A48400237A4A13806376744B1422A0
S3150800B63C83F82F20734B28221A80714B502283F8DB
S3150800B64C2E20227A6E4B83F82A20627A83F82B20D6
S3150800B65CA27A83F82C20E27A83F82D20227B83F8B1
S3150800B66C2620627B83F82720A27B83F82820E27B9E
S3150800B67C83F829200622DA75A2885A84E2889A84E5
S3150800B68C614A1188598352889A832288DA83628898
S3150800B69C1A84637E13F0100F00F03485584B002281
S3150800B6AC83F8312083F83020554C4023A375554B2D
S3150800B6BC1B881A0A22746374002384F8353084F8BC
S3150800B6CC343084F8323084F83330FFF725FFC04322
S3150800B6DC6086F2E04F4AD3780133DBB2D37063B994
S3150800B6EC93780133DBB293703BB953780133DBB2F1
S3150800B6FC537013B91378013313700023414A13801E
S3150800B70C434A1380637E052B18BF072B09D1A37EEA
S3150800B71C0133DBB2A376782B7FF470AF0023637604
S3150800B72C6CE7002B3FF46AAF228A002A74D0A27EFB
S3150800B73C511EA176002A7FF461AFE27E082A27D033
S3150800B74C591EC9B2012921D91046042A28BF04203A
S3150800B75C03218140A1760132E27603F00F03013B07
S3150800B76C072B3FF64BAF01A252F823F039BC000861
S3150800B77CB5B70008F1B70008EDBE000809B6000811
S3150800B78CEDBE000809B60008EDBE0008052ADBD197
S3150800B79C002363761D4B80221A70FCF7D7FF184BD3
S3150800B7AC142283F82F2045E7154B002283F82F2007
S3150800B7BC134B93F82F2042F0020283F82F20022213
S3150800B7CC83F83620042283F83720062283F838209B
S3150800B7DC0A2283F839200B4A2C211180602283F81F
S3150800B7EC2E202EE7094B04221A70FCF7AFFFE2E372
S3150800B7FC88330020F2330020843300207433002071
S3150800B80CBC33002070330020B83300207C33002072
S3150800B81CFE3900208801002003F00F03032B7FF468
S3150800B82CEDAEAC4B08221A70FCF790FFF4E6AA4B67
S3150800B83C1B689B88002B3FF4E1AE0023A74A1360D4
S3150800B84CA74AA8490A60A8490A60A84A1380A84AC0
S3150800B85C1380A04B08221A70FFF768FDA34B1A88B1
S3150800B86C002A3FF4CBAE02F11C0189B2A04B198019
S3150800B87CA04B080A1874597497490968087A987578
S3150800B88C1120D875083292B2100A40EA0222DA84DC
S3150800B89C002283F8282083F829208A885A84CA88A3
S3150800B8AC9A84954A1088588352889A830A88DA8328
S3150800B8BC4A881A8436338B4A13608E4C4523A373F5
S3150800B8CC0022E273627522758C490B8801339BB290
S3150800B8DC0B80190AA174E37422766276FFF7EEFDE3
S3150800B8ECC04320837B4B00221A708CE60833814AAE
S3150800B8FC938474E61C3D7E4B1D80774B804A1A60F8
S3150800B90C0EE01A880AB9598829B34FF6FF718A428C
S3150800B91C1ED07849498B8A422DD040336E4A136023
S3150800B92C6D4B1B68774A9342BFF468AE9A88002A17
S3150800B93CF3D07049898C8A42EFD1DA88002AE0D094
S3150800B94C6C49498C8A42DCD0B2F58A4FE5D1D8E7E6
S3150800B95C58888842DDD10023604A13605D4A02216B
S3150800B96C11705F4A5F490A605F490A605F4A138033
S3150800B97CFFF7DCFC72E75F4A918B5A889142CCD16F
S3150800B98CE9E7FFF7C9FD4FF6FF7398427FF436AE29
S3150800B99C5D4C5D4B9C425AD9564B93F82F3003F0AD
S3150800B9AC3F03022B7FD0534B93F82F3013F0040F21
S3150800B9BC7FF424AE4F49142381F82F304C4B2822A0
S3150800B9CC1A80502381F82E3091F8290091F82D30E1
S3150800B9DC81F8293091F8282091F82C3081F82830F4
S3150800B9EC81F82C2091F8273091F82B4081F82740C4
S3150800B9FC81F82B3091F82640444D2C7091F82A503A
S3150800BA0C81F8265081F82A400130C0B281F82D0001
S3150800BA1C60B90132D2B281F82C203AB90133DBB2C3
S3150800BA2C81F82B3013B9013481F82A40314B5A8CE2
S3150800BA3C37490A80998C59849A845A8BDA839A8B5B
S3150800BA4C1A842D4A1188598352889A832CE6617E6A
S3150800BA5C21B1284B9A8CA3889A4201D01E3498E7B8
S3150800BA6C244B5A8CE3889A42F8D1224B5A8B23885A
S3150800BA7C9A42F3D11F4B9A8B63889A42EED1174B95
S3150800BA8C1C60144B00221A701A4B93F82F2012F0D4
S3150800BA9C040F00F0DA80002363760E4B20221A700E
S3150800BAACFCF754FEAAE5134B9B8C99B2184A1380E3
S3150800BABC164B00221A70154B1B78002B7FF473AFAC
S3150800BACC144A32F81320914226D001330F4A1370C8
S3150800BADCF1E700BF7C330020803300208833002038
S3150800BAECE63300208433002074330020FE3900200E
S3150800BAFC70330020BC330020B833002086010020A8
S3150800BB0C003A0020403A00208C33002084010020A3
S3150800BB1C8E010020AC33002000249A4B1C700BE0DD
S3150800BB2C194699481E2202FB0302527E4AB1072A7D
S3150800BB3C56D00133934A1370924B1B78002BEFD0D7
S3150800BB4C02E01E2404FB0104002C3FF457AD8F4B76
S3150800BB5C1C600323A37623760023A3750422E275BF
S3150800BB6CE3768B4DAB8CA3806B8CE3806B8B23803D
S3150800BB7CAB8B638001206076864B1A7822735A78D1
S3150800BB8C62739A78A273DB78E373208295F829306E
S3150800BB9CE37295F82830A37295F82730637295F8F6
S3150800BBAC26302372FFF714FC95F82E0000F0F003EC
S3150800BBBC502B3BD9734B00221A70724B1B781A46C2
S3150800BBCC01090539B3EB810F30DA03F13601704DF3
S3150800BBDC695C59B3012911D101336A4A1370ECE730
S3150800BBEC3CB169491E2202FB0312917EA27E914248
S3150800BBFC9FD91E24644A04FB03249AE702291AD106
S3150800BC0C03F13701624D695C042914D102F138013C
S3150800BC1C695C3932AB5C43EA01235F4A138040F214
S3150800BC2C0A62934228BF13466382A382584B10229A
S3150800BC3C83F82F20BCE503F1370255498A5C002AA4
S3150800BC4CF4D013444F4A1370B7E7514B93F82E3080
S3150800BC5C1B099B004B480370EB1A9BB2143B9BB217
S3150800BC6C4E48038001F00F01022903D102F03F016F
S3150800BC7C12290FD013B912F0030F0BD0444BD98CE1
S3150800BC8C2389994240F0E781414B198D6389994282
S3150800BC9C40F0E18112F0100F47D0218A002944D0D8
S3150800BCAC04F10C00FFF766FB394B93F82A303C4A33
S3150800BCBC1078834239D1364B93F82B3051788B4216
S3150800BCCC33D1334B93F82C30927893422DD1304B99
S3150800BCDC93F82D50324BDB789D4226D12073617335
S3150800BCECA273E373E37ECBB9237EA27E9B1ADBB2E7
S3150800BCFCA17DA3EBD103DBB25AB21944C9B2A17523
S3150800BD0C002A01DA5B425AB2E07DA2EB900350FAA4
S3150800BD1C83F3DBB2E37503EBD1032376214B0122C4
S3150800BD2C1A70237EA37600232382617E01F00F030B
S3150800BD3C013B072B3FF662ACDFE813F0080038002E
S3150800BD4CAC007001BA01D8018D016101154B1B7845
S3150800BD5C13F0010F3FF452AC03236376114B4022C8
S3150800BD6C1A70002323820D4B188820B10D4B4222E2
S3150800BD7C1A70FFF72DFB0C4B00221A80FCF7E6FC19
S3150800BD8C4AE400BF840100208C330020883300204D
S3150800BD9CBC330020880100208E010020703300205F
S3150800BDAC783300207C330020FE390020AD4B1B78FD
S3150800BDBC13F0010F64D0AC4B93F82F3003F03F030C
S3150800BDCC122B5DD1A84B93F82E0000F0F003502BE4
S3150800BDDC2DD9A64B00221A70A44B1B781A460109BA
S3150800BDEC0539B3EB810F22DA03F136019E4D695CF6
S3150800BDFCE9B1012903D101339C4A1370ECE70229F6
S3150800BE0C34D103F13701984D695C04292ED102F11E
S3150800BE1C3801695C3932AB5C43EA0123944A1380D6
S3150800BE2C40F20A62934228BF13466382A382032315
S3150800BE3C63768D4B93F82620227293F8272062722C
S3150800BE4C93F82820A27293F82930E3720120FFF7A1
S3150800BE5CBFFA844B42221A7000232382854A138028
S3150800BE6C854A1380FCF772FCFFF7D6BB03F1370241
S3150800BE7C7D498A5C002ADAD013447C4A1370ABE7F6
S3150800BE8C784B20221A70FCF761FC7C4B1B6800224D
S3150800BE9C5A7688E5744B93F82F3013F0010F25D09A
S3150800BEAC11F0100F22D1238A002B7FF4A7AB714D0A
S3150800BEBC2888013080B2FFF78BFA6A4A137843F068
S3150800BECC100313702A881AB143F00203654A1370DB
S3150800BEDCFCF73CFC01232382082363760023E376D4
S3150800BEEC614B112283F82F20FFF7A4BB13F0200F08
S3150800BEFC0FD05D4890F834301A0290F8353042EA83
S3150800BF0C03065F4D2868304428605A480288931BFC
S3150800BF1C0380584B188848B111F0100F06D1514AB6
S3150800BF2C137843F002031370FFF752FA4E4B93F84B
S3150800BF3C302093F8313003EB02239BB24C4A138022
S3150800BF4CA28A934200D80BB9494B1A80484B1B88D6
S3150800BF5C6382444B1B7813F0030F3FF44FAB464BED
S3150800BF6C00221A80FCF7F2FBFFF756BB13F0100FF2
S3150800BF7C0DD00023404A13800122228204226276C5
S3150800BF8CE376394B112283F82F20FFF753BB3A4A35
S3150800BF9C128872B113F0010F01D000232382238A71
S3150800BFACDBB9638A9A4201D9334A1380324B1B8810
S3150800BFBC23820023E376334B1A68314B1A602E4BD7
S3150800BFCC1B886BB1238A5BB128332A4A1380264B0C
S3150800BFDC182283F82F20FFF730BB274A1380E8E78F
S3150800BFEC204B1B7813F0020F3FF408AB214B282289
S3150800BFFC1A801D4B102283F82F20FFF71EBB194BF6
S3150800C00C1B7813F0010F3FF4F9AA00236376154B3E
S3150800C01C10221A70FCF79AFBFFF7F0BA154B188822
S3150800C02C08B1FFF7D5F9104B93F82F3013F0010F21
S3150800C03C2DD00C4B1B7813F0010F25D007236376F4
S3150800C04C0023A37623820120FFF7C2F9054B1022A1
S3150800C05C1A70FCF77BFB044B102283F82F20FFF792
S3150800C06CE9BA00BF7C330020BC33002084010020D1
S3150800C07C8E01002070330020FE3900208833002002
S3150800C08C843300207433002006236376DBE7224BC7
S3150800C09C1B7813F0010F05D0052363760023238242
S3150800C0ACFFF7ACBA1D4B1B88002BD4D1FFF7A6BAE9
S3150800C0BC1A4B188808B1FFF78BF9194B93F82F30E0
S3150800C0CC13F0010F0CD0072363760023A376012007
S3150800C0DCFFF77EF9104B10221A70FCF737FBBAE7FC
S3150800C0EC0E4B1B88002BB6D1FFF788BA0A4B1B7868
S3150800C0FC13F0010F3FF482AA072363760023A37675
S3150800C10CFFF77CBA064B062283F830200A2283F8FE
S3150800C11C3120FFF7C9BA00BF7C33002070330020EA
S3150800C12CBC330020F8B505460E46234A138801335E
S3150800C13C9BB21380B3F5FA4F03D313464FF48052D0
S3150800C14C1A801E4B00221A701C4B1C786CB91C4B9F
S3150800C15C03EB84139F88184B1888FFF7A9F98742B5
S3150800C16CE3D00134154B1C70EEE700221A70134B02
S3150800C17C1B7863B9124A02EB831292881AB10133FF
S3150800C18C0E4A1370F3E70E4800EB831000E000200C
S3150800C19C68B1094B1A88130A43EA02238380C680BE
S3150800C1AC35B12B8803806B88438040230372F8BD16
S3150800C1BC00230360F9E700BF8C01002084010020EE
S3150800C1CC003A002000290CDD08B58AB2054B1A8006
S3150800C1DC054B1B68834203D00146184600F01BFA30
S3150800C1EC08BD7047FE39002074330020F0B43A4B72
S3150800C1FC00221A70394E02E00133374A1370364B57
S3150800C20C1B78072B18D8354D5A001A4494002E194A
S3150800C21C2A5B002AF0D07488002CEDD00588AA4237
S3150800C22CEAD142889442E7D10C68746089883181D6
S3150800C23C2B4B1B78B37222E0274B00221A7002E0B4
S3150800C24C0133254A1370244B1B78072B0AD8234D28
S3150800C25C5A001A4494002E192A5B002AF0D17288C7
S3150800C26C002AEDD1082B0CD00268334643F8042B70
S3150800C27C0A6872608A889A80194B1B78B372F0BC6C
S3150800C28C70470023174A1370174A1370124A137013
S3150800C29C02E00133104A13700F4B1B78072B11D889
S3150800C2AC0F4A147803EB430295000C4A2A44927AF7
S3150800C2BCA61A0C4D2D78AE42EBDD0A4A16700A4AC0
S3150800C2CC1370E6E7084B1B78034A137003EB43031A
S3150800C2DC9A00024E1644C7E7FA010020980100207E
S3150800C2ECF801002000020020F901002010B4164BBA
S3150800C2FC1C780134E4B21C70144B00221A7002E04C
S3150800C30C0133124A1370114B1B78072B18D8104897
S3150800C31C5A001A4491004218415A52880A43EFD0DF
S3150800C32C03EB4302910002460A44927AA21A772A30
S3150800C33CE6DD03EB43018A00014600208850DFE75F
S3150800C34C5DF8044B704700BFF8010020FA01002085
S3150800C35C98010020324B1B88292B0CD910B5304B71
S3150800C36C00221A802F4B9B8AB3F5807F07D0B3F532
S3150800C37C007F43D010BD2A4B00221A807047294BE8
S3150800C38CDA8C294B1B889A42F4D1264B1A8D264BEC
S3150800C39C5B889A42EED1254C2146A01DFFF726FF55
S3150800C3AC002204F8022C022204F8012C2168C4F895
S3150800C3BC0A10A188E1811E49086820608988A18035
S3150800C3CC44F8100C24F80C1CD4F80A1044F8161C63
S3150800C3DCE28924F8122CE288228222896282124A85
S3150800C3EC1188E18052882281082204F80A2C062238
S3150800C3FC04F8092C0A4B2A221A80BBE7094BDA8C5B
S3150800C40C094B1B889A42B5D1064B1A8D064B5B888D
S3150800C41C9A42AFD1054801460630FFF7E7FEA9E771
S3150800C42C70330020BC330020B8330020D2330020F0
S3150800C43C9001002030B4494BDA8B4FF6FF739A42C1
S3150800C44C1AD0474B1B88474909885340194208D1CB
S3150800C45C424B198C424B5B88424840884B401842E9
S3150800C46C17D0414B414A1188198052885A80404B43
S3150800C47C00221A703F4D13E0384B198C4FF6FF7398
S3150800C48C9942DED1354B3C4A1068186092889A80DE
S3150800C49C21E0354B1A805980E9E70133344A137089
S3150800C4AC334B1B78072B0ED832485A001A44910086
S3150800C4BC45182D4A1488425A9442EED12A4A508875
S3150800C4CC6A889042E9D1082B16D0244B55F8042FCC
S3150800C4DC1A60AA889A80214B284A1168C3F8061054
S3150800C4EC92885A8108221A7300225A73244A13888E
S3150800C4FC0E33138030BC7047184B4FF0FF321A605E
S3150800C50C9A8000221A629A841C490868C3F80600A5
S3150800C51C89885981C3F81600598313490888D88421
S3150800C52C498819850E49088898834988D9831A75C4
S3150800C53C012159759A73D973082119745A740622EC
S3150800C54C9A740422DA74197306225A7336330D4A0E
S3150800C55C13600B4B2A221A80CCE700BFBC33002091
S3150800C56CB8330020B4330020FC010020B03300207F
S3150800C57CFA0100209801002080C6000890010020CE
S3150800C58C703300208433002010B504464160FEF752
S3150800C59C88FB206010BD10B50446FEF782FB2368A5
S3150800C5ACC01A63689842B4BF0020012010BD000071
S3150800C5BC70B50D4E0D4CA41BA4100025A54209D12F
S3150800C5CC0B4E0C4C00F03AF8A41BA4100025A542FF
S3150800C5DC05D170BD56F8253098470135EEE756F863
S3150800C5EC253098470135F2E790C6000890C6000832
S3150800C5FC90C6000894C6000830B50024A24201D1A2
S3150800C60C002007E0035D01340D1915F8015CAB42F7
S3150800C61CF4D0581B30BD10B5431E0A44914200D1C4
S3150800C62C10BD11F8014B03F8014FF7E70244034616
S3150800C63C934200D1704703F8011BF9E7F8B500BF20
S3150800C64CF8BC08BC9E467047F8B500BFF8BC08BCD9
S3090800C65C9E46704731
S3150800C6600000000000000000010203040607080994
S3150800C670000000000102030463825363ADDE122347
S30D0800C680FFFFFFFFFFFF0000AA
S30D0800C688E4BBFF7F010000007E
S3090800C69021820008ED
S3090800C694FD8100080E
S3110800C6980024F40001000000100000005F
S70508008CFD69
